:100000000C942A001895000018950000189500001F
:10001000189500001895000018950000189500002C
:10002000189500001895000018950000189500001C
:10003000189500001895000018950000189500000C
:1000400018950000189500001895000018950000FC
:10005000189500008FE58DBFC0E2ECEA4E2E84E0DB
:100060008EBFD4E0F3E05F2EEEEFF3E0A0E6B0E069
:1000700088278D933197E9F76624899A9198889813
:100080008D9A8C988E9A9598ADE7B0E0ECEDFBE0F8
:100090000E941A05A1E8B0E0E0EEFBE00E941A051C
:1000A000E1E8F0E00E94DC03EDE7F0E00E94D70316
:1000B0000E944C04FF27EDE0A5E8B0E00E94E805AF
:1000C000ECEEFBE00E94AE020E94B60280E090E0FF
:1000D000A9E8B0E08D939C9381E080938B00009120
:1000E0008B000C3018F011F00C94BA009598BB27D7
:1000F000A0E38C9184FBDEF383E090E00E94DB02BE
:1001000080E090E0AFE6B0E08D939C93969A959A4C
:100110000027BB27A0E38C9184FB0EF401E041E0B3
:10012000041710F00C94A200AFE6B0E00D911C9102
:1001300041E050E0040F151FAFE6B0E00D931C93B3
:100140000C94880095989698A9E8B0E00D911C91C0
:10015000AFE6B0E04D915C91040F151FA9E8B0E047
:100160000D931C93ABE8B0E08C918F5F8C9310F4EF
:100170000C946F00A9E8B0E00D911C914CE050E0A8
:100180000E941B02A9E8B0E04D935C93E6E1FCE01D
:100190000E94AE02A4E9B3E0E9E8F0E00E948A051B
:1001A0000E94BA02A9E8B0E00D911C9122273327E2
:1001B000A1E7B0E04D915C91662777270E94770513
:1001C000ABE6B0E00D931D932D933D93ABE6B0E00D
:1001D0000D911D912D913C91A3E7B0E04D915C9163
:1001E000662777270E947705ABE6B0E00D931D9355
:1001F0002D933D93ABE6B0E00D911D912D913C9177
:10020000A5E7B0E04D915C91662777270E947705BE
:10021000ABE6B0E00D931D932D933D93ABE6B0E0BC
:100220000D911D912D913C91A7E7B0E04D915C910E
:10023000662777270E947705ABE6B0E00D931D9304
:100240002D933D93ABE6B0E00D911D912D913C9126
:10025000A9E7B0E04D915C91662777270E9477056A
:10026000ABE6B0E00D931D932D933D93ABE6B0E06C
:100270000D911D912D913C91ABE7B0E04D915C91BA
:10028000662777270E947705ABE6B0E00D931D93B4
:100290002D933D93ABE6B0E00D911D912D913C91D6
:1002A00047E050E060E070E00E943802ABE6B0E06A
:1002B0004D935D936D937D93EEE1FCE00E94AE0261
:1002C000A4E9B3E0EBE6F0E00E948D050E94BA02DB
:1002D000A9E7B0E08D919C91ABE7B0E08D939C9342
:1002E000A7E7B0E08D919C91A9E7B0E08D939C9336
:1002F000A5E7B0E08D919C91A7E7B0E08D939C932A
:10030000A3E7B0E08D919C91A5E7B0E08D939C931D
:10031000A1E7B0E08D919C91A3E7B0E08D939C9311
:10032000A9E8B0E08D919C91A1E7B0E08D939C93FA
:10033000E4EEFBE00E940D05EBE6F0E00E94D7033F
:100340000E94FB030E94A304FF27EDE0ACE8B0E0AD
:100350000E94E805EBE6F0E00E94D7030E94FB0351
:10036000A3E6B0E00E942C04E5E8F0E00E94DC0384
:10037000ECE8F0E00E94D7030E944C04FF27EDE078
:10038000A0E9B0E00E94E805E0E9F0E00E94DC03AB
:10039000E8EEFBE00E9404050E94B204FF27EDE0B6
:1003A000A4E9B0E00E94E805E4E2FCE00E94AE02AD
:1003B000A4E9B3E0AF93BF93E4E9F0E00E94D70370
:1003C0000E94EA0211E001E0BF91AF910E942F0567
:1003D000E4E9F3E0A4E9B3E00E94E3050E94BA0275
:1003E0000E94B60284EF91E00E94DB020C9466004A
:1003F00000FC10D0089503D01ED001F8F9CF0024DE
:10040000E89457FF02C009D0689400F80BD010F8A8
:100410000124089502D009D00895509540954F5F6A
:100420005F4F0895E89417FF0895009510950F5FAA
:100430001F4F68940895352F242FE894452B11F40D
:1004400068940895512F402F0027112780E1440F11
:10045000551F001F111F021B130B416018F4020FE0
:10046000131F4E7F8A9599F7089500FC05D00895D3
:1004700030D005D001F8F9CF37D03FD00895842F80
:10048000952FA62FB72FE894452B462B472B11F419
:1004900068940895402F512F622F732F0027112742
:1004A00022273327F0E2440F551F661F771F001FD6
:1004B000111F221F331F081B190B2A0B3B0B416016
:1004C00028F4080F191F2A1F3B1F4E7FFA9559F772
:1004D00008950024E89477FF02C006D0689400F8DD
:1004E00009D010F80124089512D04F5F5F4F6F4F6D
:1004F0007F4F0895E89437FF089500951095209553
:1005000030950F5F1F4F2F4F3F4F689408954095D0
:1005100050956095709508953197F1F70895689416
:1005200062F80895E89462F808958F939F9383E6A4
:1005300090E00197F1F79F918F91089580952AE0BF
:1005400090E0089410F0919802C0919A0000EDDFBD
:10055000ECDF969587952A95A9F70895C895802D83
:10056000882319F0EBDF3196F9CF08958DE0E6DFAF
:100570008AE0E4CFA4E9B3E08D91882311F0DEDFB7
:10058000FBCF08958F939F9383E690E00197F1F757
:100590009F918F91089529E0809BFECFF3DFF2DFDA
:1005A000F1DF8894809908942A9519F0879597959A
:1005B000F6CF80950895EF93FF93EE27E82BE92B74
:1005C00031F0E0EDF7E03197F1F70197D1F7FF91C6
:1005D000EF9108958DE207FD8D938F2D881F802F59
:1005E000881F8F57082F6894F7F8802F87FF15C052
:1005F00080958395082F80E38D938EE28D93802FD5
:10060000815228F080E38D9399279C930895442785
:100610000A95802F09F196D01FC0805230F09EE4D9
:100620009D9381E48D939D93EFCF4427DF92EF92CA
:10063000FF920F938FE1801B11F0082F83D089D098
:100640009EE29D930F91FF90EF90DF9044270395DA
:10065000003209F4D7CF2BD03F93E4EEF6E038E137
:100660002F2D1E2D0D2DFF24EE24DD244427000FF9
:10067000111F221FA8F42F923F920E940005102CF8
:100680000E940005202C0E940005302C0E940005CD
:100690003197410DD21CE31CF01C3F902F9001C0FC
:1006A000339631963A9519F73F9107D0AFCFDD0CCD
:1006B000EE1CFF1C0A95D9F70895002719E058D0C1
:1006C0008F93802B11F0039501C08F911A95B9F784
:1006D000802F882309F496CF8F91805D8D930A95A2
:1006E000D9F792CF0065CD1D80B2E60E4059730751
:1006F000A0ACB90350D6DC01286BEE00943577002E
:10070000CA9A3B0065CD1D00B2E60E005973070082
:10071000ACB90300D6DC01006BEE000035770000B9
:100720009A3B0000CD1D0000E60E0000730700009C
:10073000B9030000DC010000EE00000077000000BB
:100740003B000000F694E794D79447950A95D1F7BB
:10075000089500270DD08F9303958F2D8E298D2915
:10076000842BC1F78F91805D8D930A95D9F74CCF7B
:100770001F930F93002710E2440FDD1CEE1CFF1C9B
:10078000001F802F9AE0890B10F0082F43951A95CF
:1007900099F7802F0F911F910895D094E094F094D1
:1007A00091E0D90E9927E91EF91E10950895D19070
:1007B000E190F190019108952191319141915191F0
:1007C0000895102F90E8FF0C001F0927990FF79448
:1007D0001078652F90E8440F551F5927990F4795BA
:1007E000607800380895FF0C90E89027110F9795D6
:1007F000F794092F0895102FBD2CDE2CEF2CF02E2E
:1008000011234AF4B094D094E094F0949FEFB91A75
:10081000D90AE90AF90A0EE1FF2039F4FE2CED2C81
:10082000DB2CBB240850C2F76BC032F00A95BB0C1E
:10083000DD1CEE1CFF1CF9CF01D0D5CFB7FE08950B
:1008400090E8B91611F4D0FE08959FEFD91AE90A7D
:10085000F90A09F403950895DD92ED92FD920C9347
:100860000895502F2D2D3E2D4F2D612F08952DECE5
:100870003CEC4CEC5DE366270FC099DFF2DFDD2432
:10088000EE2490E8F92E0FE307C096DF05C022277B
:10089000332740E251E46627552351F1002381F1CB
:1008A00090DF71F11627005850580894050B18F482
:1008B00007FD03C025C007FD23C046953795279542
:1008C000F694E794D79422D0FF202AF0DD0CEE1C9A
:1008D000FF1C015073F09D2D969548F0DD203AF4F1
:1008E000EE202AF491E0D90E9927E91EF91E7BCF5C
:1008F00007C09FE7092FF92A9FEFD92EE92E089507
:10090000DD24EE24FF240027112708959F929924C7
:10091000AA24BB2488E1D216E306F40628F0D21AF2
:10092000E30AF40A089401C08894991CAA1CBB1C11
:10093000DD0CEE1CFF1C8A9571F7D92CEA2CFB2CE0
:100940009F90089539DF3DDF503829F090E86927FE
:100950000CC00AF045D047CF5FE322273327442756
:1009600001C02ADF2EDF5038B1F3003899F3902F01
:10097000951B8BF312F434D0FACF983118F022275C
:1009800033274427983028F0232F342F44279850BA
:10099000F9CF992329F04695379527959A95D9F758
:1009A000912F962742F014D0B0F6F794E794D7949D
:1009B0000F5F8BF69ECF10D051F008F4EEDEFF20D3
:1009C00052F2DD0CEE1CFF1C0150CBF792CF98CFFA
:1009D000D20EE31EF41E0895D21AE30AF40A089513
:1009E000DF92EF92FF920F931F93D22EE32EF42EFD
:1009F000052F162F6F915F914F913F912F91089581
:100A0000C895319600200895FBDFD02CF9DFE02C4B
:100A1000F7DFF02CF5DF002D0895F2DF202DF0DF59
:100A2000302DEEDF402DECDF502D089591E005C014
:100A300092E003C094E001C098E0E2DF0D929A9545
:100A4000E1F7089599278D9193958823E1F7939580
:100A500011968C9311978E919A95D1F70895EA2F5C
:100A6000FB2F00244C918D9103948E32E1F71124D9
:100A70008D9113948823E1F71A94101640F411977E
:100A8000202F2119239580E38D932A95E9F71130C2
:100A900039F59927AE2FBF2FA00DB91FA00FB91F91
:100AA0008C919C93853308F421C031E08E918E3275
:100AB000E9F38D3241F0830F8A3319F480E331E09A
:100AC00001C033278C93AE1789F7332341F0AE2F43
:100AD000BF2FB8DF81E34D3209F43196808308954A
:100AE0008827E00DF81FE00FF81F80830895040F9A
:100AF000151F261F371F0895000F111F221F331FB8
:100B0000089500951095209530950F5F1F4F2F4F3A
:100B10003F4F0895019110810EC0019111912191D3
:100B200030810BC00191108117FF05C03FEF2FEFFF
:100B300004C0008111272227332737FF03C0E1DFDC
:100B40008DE28D93CF93DF93CF92DF92EF92AA2421
:100B5000BB24CC24DD24EE2440E2CAE0DD2755E0AE
:100B600093E38881890F87FD9F7083FD907F891BA8
:100B700089935A95A9F7C0DFAA1CBB1CCC1CDD1CAD
:100B8000EE1C4A9551F7E894EFE0FF2782910ED0D2
:100B9000EB30E0F71EF068948A2D0CD088278D93F7
:100BA000EF90DF90CF90DF91CF910895982F8295AD
:100BB00001D0892F8F70805D26F0803309F408956D
:100BC00068948D93089581918D938823E1F708951A
:100BD00094E081918D939A95E1F708950000084281
:100BE0000000F84100E08444000030426D313638A6
:100BF0002D746573742D636170616369746F722DF8
:100C000072632D74696D696E672D646972656374B2
:100C10002E626173000074776F72643D0000206182
:0C0C200076673D002025206176673D00CE
:00000001FF
